:020000040000FA
:100000000002040000000000D4020000D40200003E
:10001000D4020000D4020000D4020000D402000088
:10002000D4020000D4020000D4020000D402000078
:10003000D4020000D4020000D4020000D402000068
:10004000D4020000D4020000D4020000D402000058
:10005000D4020000D4020000D4020000D402000048
:10006000D4020000D4020000D4020000D402000038
:10007000D4020000D4020000D4020000D402000028
:10008000D4020000D4020000D4020000D402000018
:10009000D4020000D4020000D4020000D402000008
:1000A000D4020000D4020000D4020000D4020000F8
:1000B000D4020000D4020000D4020000D4020000E8
:1000C000D4020000D4020000D4020000D4020000D8
:1000D000D4020000D4020000D4020000D4020000C8
:1000E000D4020000D4020000D4020000D4020000B8
:1000F000D4020000D4020000D4020000D4020000A8
:10010000D4020000D4020000D4020000D402000097
:10011000D4020000D4020000D4020000D402000087
:10012000D4020000D4020000D4020000D402000077
:10013000D4020000D4020000D4020000D402000067
:10014000D4020000D4020000D4020000D402000057
:10015000D4020000D4020000D4020000D402000047
:10016000D4020000D4020000D4020000D402000037
:10017000D4020000D4020000D4020000D402000027
:10018000D4020000D4020000D4020000D402000017
:10019000D4020000D4020000D4020000D402000007
:1001A000D4020000D4020000D4020000D4020000F7
:1001B000D4020000D4020000D4020000D4020000E7
:1001C000D4020000D4020000D4020000D4020000D7
:1001D000D4020000D4020000D4020000D4020000C7
:1001E000D4020000D4020000D4020000D4020000B7
:1001F000D4020000D4020000D4020000D4020000A7
:10020000FFFFFF00FFFFFF00D4020000D402000048
:10021000D4020000D4020000D4020000D402000086
:10022000D4020000D4020000D4020000D402000076
:10023000D4020000D4020000D4020000D402000066
:10024000D4020000D4020000D4020000D402000056
:10025000D4020000D4020000D4020000D402000046
:10026000D4020000D4020000D4020000D402000036
:10027000D4020000D4020000D4020000D402000026
:10028000D4020000D4020000D4020000D402000016
:10029000D4020000D4020000D4020000D402000006
:1002A000D4020000D4020000D4020000D4020000F6
:1002B000D4020000D4020000D4020000D4020000E6
:1002C000D4020000D4020000D4020000D4020000D6
:1002D000D4020000D4020000D4020000D4020000C6
:1002E000D4020000D4020000D4020000D4020000B6
:1002F000D4020000D4020000D4020000D4020000A6
:10030000D4020000D4020000D4020000D402000095
:10031000D4020000D4020000D4020000D402000085
:10032000D4020000D4020000D4020000D402000075
:10033000D4020000D4020000D4020000D402000065
:10034000D4020000D4020000D4020000D402000055
:10035000D4020000D4020000D4020000D402000045
:10036000D4020000D4020000D4020000D402000035
:10037000D4020000D4020000D4020000D402000025
:10038000D4020000D4020000D4020000D402000015
:10039000D4020000D4020000D4020000D402000005
:1003A000D4020000D4020000D4020000D4020000F5
:1003B000D4020000D4020000D4020000D4020000E5
:1003C000D4020000D4020000D4020000D4020000D5
:1003D000D4020000D4020000D4020000D4020000C5
:1003E000D4020000D4020000D4020000D4020000B5
:1003F000D4020000D4020000D4020000D4020000A5
:100400000F8020000E7F22000E01880000000000F7
:100410000C000700802D20000100200011000700C3
:10042000000020000000E000020032000000020096
:100430000000000090020200000000000040DA000E
:100440000000FE004440A900000020000000E00081
:100450000300320000002000A00188004440A800F2
:100460000000060091018800800078000000EB0089
:1004700015003700E280400032A0B4009101BA00BC
:10048000E280400032A0B4009102BA00E280400055
:1004900032A0B4000002EB00472BDE00F507B200EB
:1004A000602CE10004003A000059EB008301E900F0
:1004B000FDFF3E00040037006128E100010032002A
:1004C0000082EB00040007001101BA000200E00006
:1004D000E8FF3A00000006003159BA008301E90044
:1004E0000C0032002159BA008301E90008003200F3
:1004F0000400E00003003A00E280400032A0B400B3
:10050000F5FF370011D9BA008301E900FAFF3A007C
:100510008100E800E180400032A0B4000000060045
:100520000400FA004507A9000080EB00601988006C
:100530004227A900C022A900C422A900C4C2BF004A
:100540000080FB000000D1006140600000C0EA00B4
:10055000614060006140600000414000412C20008B
:1005600091407800D0CFB30000C06000024070001E
:10057000C4E2B700F0FF2F00F1002000008FBE00A2
:100580000080EB008080EB001E0F40005E9748006B
:100590000080EB008080EB00BE0F1000AE8F1800D3
:1005A000F7FF3A00E5FF37000040DA000000FE00E8
:1005B00000000000FFFFFF00FFFFFF00FFFFFF0044
:1005C000FFFFFF00FFFFFF00FFFFFF00FFFFFF0037
:1005D000FFFFFF00FFFFFF00FFFFFF00FFFFFF0027
:1005E000FFFFFF00FFFFFF00FFFFFF00FFFFFF0017
:1005F000FFFFFF00FFFFFF00FFFFFF00FFFFFF0007
:020000040001F9
:00000001FF
